:020000021000EC
:10F800000C9446FC0C9463FC0C9463FC0C9463FC19
:10F810000C9463FC0C9463FC0C9463FC0C9463FCEC
:10F820000C9463FC0C9463FC0C9463FC0C9463FCDC
:10F830000C9463FC0C9463FC0C9463FC0C9463FCCC
:10F840000C9463FC0C9463FC0C9463FC0C9463FCBC
:10F850000C9463FC0C9463FC0C9463FC0C9463FCAC
:10F860000C9463FC0C9463FC0C9463FC0C9463FC9C
:10F870000C9463FC0C9463FC0C9463FC0C9463FC8C
:10F880000C9463FC0C9463FC0C9463FC11241FBE69
:10F89000CFEFD0E1DEBFCDBF11E0A0E0B1E0EEE9F7
:10F8A000FFEF01E00BBF02C007900D92A430B1073B
:10F8B000D9F712E0A4E0B1E001C01D92A634B1076F
:10F8C000E1F70C9491FF0C9400FC0F92AF93BF935F
:10F8D000CF93DF93EF93FF93FC01EA01DB01D8950F
:10F8E000099231961197D9F7FF91EF91DF91CF915E
:10F8F000BF91AF910F9008950F921F920F93AF9306
:10F90000BF93CF93DF93EF93FF93FC01EA01DB01F9
:10F910000990199001E043D032961297C9F7FC0183
:10F9200003E03DD005E03BD0FF91EF91DF91CF9117
:10F93000BF91AF910F911F900F9008950F931F9358
:10F94000EF93FF93FC0103E02AD000E011E0E00F09
:10F95000F11FE617F707B9F7FF91EF911F910F918C
:10F9600008950F930F9222D0082E09E018D00F901F
:10F970000F9108950F930F92EF93FF9317D0FC010F
:10F9800060936800C895802DFF91EF910F900F91C3
:10F9900008950F930BD001E102D00F910895E199E2
:10F9A000FECF00936800E895FFFF0000009168001B
:10F9B00000FDFCCF089589E08093990080919A0022
:10F9C000886180939A00089580919A00877E809341
:10F9D0009A00089580939C0080919B0086FFFCCF45
:10F9E00080919B00806480939B00089580919C008F
:10F9F0009927089580919B009927807890700895A9
:10FA0000EF92FF920F931F93CF93DF937B01C0E0A0
:10FA1000D0E0C617D70770F48C010E94FAFC882347
:10FA2000E1F30E94F6FCF80181938F012196CE1537
:10FA3000DF0598F381E090E0DF91CF911F910F9166
:10FA4000FF90EF900895EF92FF920F931F93CF9343
:10FA5000DF937C018B01C0E0D0E0C017D10738F400
:10FA6000F70181917F010E94EAFC2196F6CF81E0A7
:10FA700090E0DF91CF911F910F91FF90EF9008954B
:10FA8000EF92FF920F931F93CF93DF937C0100E0DF
:10FA900010E00817190788F4C0E0D0E000000E94C9
:10FAA000FAFC882351F4219688E0CA3CD807B0F3C9
:10FAB0000F5F1F4F0E151F0578F3DF91CF911F9138
:10FAC0000F91FF90EF9008950E94E4FC0E940000C7
:10FAD0000895DF92EF92FF920F931F93CF93DF93DE
:10FAE000CDB7DEB72197DEBFCDBF8C017B01198278
:10FAF000D98061E070E0CE01860F971F0E9400FD63
:10FB000089818B31B1F761E070E0C8010E9400FD8E
:10FB100061E070E0CE01860F971F0E9400FD898191
:10FB20009927182F002761E070E0CE01860F971FFC
:10FB30000E9400FD8981080F111D61E070E0CE0177
:10FB4000860F971F0E9400FD89818E30B9F4C8018D
:10FB50000196BC01C7010E9400FD98018FEF0F3F85
:10FB6000180779F0F70181917F01D82621503040A4
:10FB7000FFEF2F3F3F07B1F7DD2019F080E090E065
:10FB800001C0C8012196DEBFCDBFDF91CF911F918B
:10FB90000F91FF90EF90DF900895CF92DF92FF9248
:10FBA0000F931F93CF93DF93182FEB016A018BE123
:10FBB0000E94EAFC4BE1F42E812F0E94EAFCF12620
:10FBC0000D2F1127802F0E94EAFCF0268C2F0E9417
:10FBD000EAFCFC268EE00E94EAFC8EE0F8262197E3
:10FBE0008FEFCF3FD80759F0F60181916F01F826CA
:10FBF0000E94EAFC2197FFEFCF3FDF07A9F78F2D87
:10FC00000E94EAFCDF91CF911F910F91FF90DF904E
:10FC1000CF90089599278139910559F0823991053E
:10FC200024F48039910529F008C08239910519F032
:10FC300004C082E003C087E001C080EC99270895EA
:10FC4000BF92CF92DF92EF92FF920F931F93CF93C9
:10FC5000DF93B82E8B01FB018081C82FDD27C231D5
:10FC6000D10509F46DC0C331D105DCF4C330D10531
:10FC700009F44DC0C430D10544F4C130D10579F147
:10FC8000C230D10509F44AC018C1C630D10509F403
:10FC90004AC0C630D1050CF410C160970CF40DC1F8
:10FCA00054C0C531D10509F4DCC0C631D10544F4D6
:10FCB000C331D10509F47CC0649709F449C0FDC083
:10FCC000CA31D10509F4EBC0CB31D10524F46697D4
:10FCD00009F4AEC0F2C06B9709F4D8C0EEC0FB01C6
:10FCE000118288E0828381E4838386E5848382E5D0
:10FCF000858389E4868383E5878380E580878FE534
:10FD0000818782E38287AB016BE070E0DCC0FB019E
:10FD100081810E940AFEF801828301C0FB011182E9
:10FD2000A801BE01D0C0FB0183819927982F8827A5
:10FD30002481820F911D909345028093440206C056
:10FD400060E070E0CB010E949EFCF8011182B8C017
:10FD5000FB0181819927D82FCC2782819927C82B35
:10FD6000D92B809144029091450297FF03C081E016
:10FD70008BBF01C01BBEF8011182C8010296209101
:10FD8000440230914502AC01BE01C901880F991FA0
:10FD90000E9465FCF801EC0FFD1F12829E01369552
:10FDA00027958091440290914502820F931F53C082
:10FDB000FB0181819927D82FCC2782819927C82BD5
:10FDC000D92B809144029091450297FF03C081E0B6
:10FDD0008BBF01C01BBECC24DD24CC16DD06D8F4BD
:10FDE000FAE0EF2EF12CE00EF11E8091440290918A
:10FDF0004502880F991FA70160E071E08C0D9D1DE1
:10FE00000E947CFC80E091E0C80ED91EE80EF91E2D
:10FE1000CC16DD0650F30E94C9FCF8011182D6957C
:10FE2000C79580914402909145028C0F9D1F29C077
:10FE3000FB0181819927D82FCC2782819927C82B54
:10FE4000D92B1182EC0FFD1F1282809144029091F8
:10FE500045028C0F9D1F9093450280934402239688
:10FE60005FCFFB0181819927382F22278281992733
:10FE7000282B392B11828091440290914502820FE8
:10FE8000931F90934502809344021AC0FB01118294
:10FE90008481E82FFF27E050FF4F808107C0FB01DE
:10FEA000118269E081E090E00E94BAFCF80182834F
:10FEB0001382A80164E070E006C089ECF801818338
:10FEC000A80162E070E08B2D0E94CDFDDF91CF9103
:10FED0001F910F91FF90EF90DF90CF90BF9008950A
:10FEE000CF93DF93CDB7DEB72197DEBFCDBF69E0FB
:10FEF00081E090E00E94BAFC992784FF09C08F7EC0
:10FF00000E94B1FC05C064E071E089810E9420FE7E
:10FF100064E071E0CE0101960E9469FD892B99F39E
:10FF2000F7CFCFEFD0E1DEBFCDBFCEE1F894AEEF9B
:10FF3000BFE00E94C6FF802D843B79F4AFEFBFE0A5
:10FF40000E94C6FF802D833C41F4ADEFBFE00E94CC
:10FF5000C6FF802D992780936F000E94DBFC0E94D2
:10FF6000F6FC84E690E00E9440FD0E94FAFC8823A3
:10FF700019F00E9470FF04C0C150C8BBCC2389F7A0
:10FF80000E9464FD80E090E00C94CEFFE199FECFEA
:0EFF9000BFBBAEBBE09A11960DB20895FFCF35
:04FF9E001E970200A8
:040000031000F800F1
:00000001FF
